:100000000C9480000C94A8000C94A8000C94A800F8
:100010000C94A8000C94A8000C94E00F0C94A80079
:100020000C94A8000C94A8000C94A8000C94A800B0
:100030000C94A8000C94C70E0C94A8000C94A80073
:100040000C94A8000C94A8000C94B9110C94A8006E
:100050000C9431130C94A8000C94A8000C94A800E4
:100060000C94A8000C94A8000C94A8000C94A80070
:100070000C94780C0C94A8000C94A80000002100AB
:10008000240027002A0000002200250028002B0061
:1000900000002000230026002900020202020202C2
:1000A000020204040404040404040303030303031A
:1000B00003030101010101010101010204081020F3
:1000C0004080010204081020408001020408102032
:1000D000408080402010080402010000000102005E
:1000E00000000000000004030706000000000000FC
:1000F00000000000000000000000F6096F10481426
:1001000011241FBECFEFD0E1DEBFCDBF11E0A0E0D4
:10011000B1E0E6EBFEE202C005900D92AA31B10714
:10012000D9F71BE0AAE1B1E001C01D92AC33B107E1
:10013000E1F710E0C0E0D1E004C02297FE010E9488
:100140002216CA3FD107C9F70E9496150C94591779
:100150000C94000089E190E090932F0280932E028E
:100160008EE190E09093310280933002109233023E
:100170001092320284E690E090933502809334022C
:1001800082E390E0909337028093360210923A0215
:1001900010923B0210923C0210923D0208954F9241
:1001A0005F926F927F928F929F92AF92BF92CF9207
:1001B000DF92EF92FF920F931F93CF93DF93EC01A7
:1001C0006A807B808C809D80A880B980CC24B7FC1D
:1001D000C094DC2CA618B708C808D9088E819F8166
:1001E000A885B985A80EB91ECA1EDB1E4C845D8485
:1001F00020912E0230912F02442737FD4095542F35
:10020000C601B5010E949D157B018C01209132022F
:1002100030913302429EC001439E900D529E900D3C
:100220001124AA2797FDA095BA2FE80EF91E0A1FE0
:100230001B1F8A859B85AA2797FDA095BA2FA6012B
:100240009501281B390B4A0B5B0BCA01B9012091A0
:10025000300230913102442737FD4095542F0E94DF
:100260009D15E60EF71E081F191F209134023091CC
:100270003502442737FD4095542FC801B7010E942D
:100280000516BB86AA866E827F82888699868E85B1
:100290009F85AA2797FDA095BA2F280F391F4A1FBF
:1002A0005B1F2F3F3105410551056CF422308FEF64
:1002B00038078FEF48078FEF580754F0A40CB51C90
:1002C000BD86AC8609C02FEF30E040E050E004C0AE
:1002D00021E03FEF4FEF5FEF3F872E87DF91CF9118
:1002E0001F910F91FF90EF90DF90CF90BF90AF9054
:1002F0009F908F907F906F905F904F900895109295
:1003000039021092380210923E0210924A02109264
:10031000490210924C0210924B0210924E0210921F
:100320004D0210925A021092590210925C021092E1
:100330005B0210925E0210925D020895EF92FF92AE
:100340000F931F9380913E02882309F460C080912F
:10035000380290913902009709F459C00E940112A5
:100360007B018C0180913A0290913B02A0913C026A
:10037000B0913D028E159F05A007B10708F047C058
:1003800080918F0A9091900AA091910AB091920A5F
:100390008093410290934202A0934302B09344029F
:1003A0008091930A9091940AA091950AB091960A2F
:1003B0008093510290935202A0935302B09354023F
:1003C0008FE392E00E94CF008FE492E00E94CF0082
:1003D0008091380290913902009761F060914D024E
:1003E00070914E0240915D0250915E0286E292E071
:1003F0000E94CF0FD801C7018196A11DB11D809326
:100400003A0290933B02A0933C02B0933D021F91AD
:100410000F91FF90EF90089585E29BE040E052EC51
:1004200061E070E00E94591360E472E48FE090E0B4
:100430000E94F30C8FE89AE00E9461100E94AA00CB
:1004400080E061E00E94FA1008956F927F928F928F
:100450009F92BF92CF92DF92EF92FF920F931F93E2
:10046000CF93DF938091880190E0C0908601DD24D6
:100470002DEF3FEFC20ED31E09E811E0EBEFBE2EC9
:10048000B80E76EE872E7FEF972E880E991E8CC0C1
:10049000C4014A96843091050CF48CC084309105D7
:1004A00029F4F80180818093CC0075C08F309105CC
:1004B000BCF4F801808181FF03C08B2D61E002C094
:1004C0008B2D60E00E941E11F801808180FF03C027
:1004D0008B2D61E002C08B2D60E00E94FA105BC0A2
:1004E0008F30910509F457C08031910529F4F80146
:1004F0008081809306014FC08131910509F44BC082
:100500008A3191050CF456C08E3291050CF052C020
:10051000F80180817401F594E79480FC08C0F7012C
:10052000EE0FFF1FEE5DFD4F8083118234C0F70197
:10053000EE0FFF1FEE5DFD4F782E66246081718106
:10054000660D771D71836083CB01855F9140F7E075
:100550008F3C9F07A0F4E701CC0FDD1FCC0FDD1F00
:10056000C65EDD4FCE010E94940ECE010E94B40EF5
:10057000882389F4CE01B7010E946B0E0CC061156F
:10058000710549F4C701880F991F880F991F865E6E
:100590009D4F0E94720E0894C108D1080F5F1F4F33
:1005A000B3940894811C911C1C141D040CF470CF8E
:1005B00080E001C080E4DF91CF911F910F91FF9007
:1005C000EF90DF90CF90BF909F908F907F906F9033
:1005D0000895CF92DF92EF92FF920F931F93DF93D4
:1005E000CF930F92CDB7DEB780918801C82EDD245E
:1005F0000091890110E0EE24FF2452C0C114D104FF
:10060000B1F131E0C316D104A1F182E0C816D104E2
:10061000B1F1E3E0CE16D10471F1F4E0CF16D104CC
:1006200061F130E1C316D10444F485E0C816D10469
:1006300011F423B125C029B123C0E0E1CE16D104C5
:1006400019F4209106011CC0F1E1CF16D104C1F0CC
:100650002AE1C216D1049CF48C2D82510E94801094
:10066000BC017595679575956795262F09C02CE295
:1006700007C021E005C02DEF03C022E201C020E049
:10068000E20EF11C85E29BE0622F40E050E02983FE
:100690000E944E150894C11CD11C015010402981A4
:1006A0000115110509F0AACFC7010F90CF91DF9175
:1006B0001F910F91FF90EF90DF90CF900895EF92F0
:1006C000FF920F931F93CF93DF931092FE09109226
:1006D000FD091CE3E12EF12C48C010E085E29BE00F
:1006E0000E94C6128834910509F451C00E9DE001A4
:1006F0000F9DD00D1E9DD00D1124C15ADD4F00E07D
:1007000010E009C00F5F1F4F499159918AE191E0B4
:10071000B8010E94050C80911C0190911D010817E1
:10072000190784F38091FD099091FE09FC01EE0FF9
:10073000FF1FE80FF91FE959F64F618172818AE1C5
:1007400091E00E94420B04C08AE191E00E948C0B70
:1007500080911A018823C1F78091FD099091FE09CB
:1007600001969093FE098093FD098091FD09909177
:10077000FE09FC01EE0FFF1FE80FF91FE959F64FC4
:1007800000810F3F09F0A9CF20E030E002C021E056
:1007900030E0C901DF91CF911F910F91FF90EF9051
:1007A0000895EF92FF920F931F93CF93DF938C01E5
:1007B0007B01C5E2DBE0CE016FEF70E040E050E08E
:1007C0000E948C15CE016FEF70E040E050E00E9477
:1007D0008C15CE01B80140E050E00E948C15CE018E
:1007E00062E070E040E050E00E948C15CE01B7015D
:1007F00040E050E00E948C15C80102968E0D9F1DAE
:1008000060E071E00E94D0156FEF70E0681B790B1B
:10081000CE0140E050E00E948C15DF91CF911F91F6
:100820000F91FF90EF9008952F923F924F925F9219
:100830006F927F928F929F92AF92BF92CF92DF92F0
:10084000EF92FF920F931F93DF93CF93CDB7DEB755
:100850002E970FB6F894DEBF0FBECDBF612C01E01E
:10086000702E13E0212E312CB5E18B2E912C4424D7
:10087000439482C580918301909184010097B9F4DB
:1008800085E29BE00E94C6128F3F910509F074C576
:1008900022E030E0309384012093830180E00E94C5
:1008A0007011642D681B80E00E941E1165C58230A6
:1008B000910571F485E29BE00E94C6128093850148
:1008C0008F3F09F459C5309284012092830154C5A9
:1008D00083309105B1F485E29BE00E94C6128093BB
:1008E00086012091850130E0280F311D30931902D7
:1008F0002093180284E090E0909384018093830118
:100900003BC584309105C9F485E29BE00E94C61284
:10091000809387012091180230911902280F311D10
:1009200030931902209318021092170245E050E00C
:1009300050938401409383011FC58530910509F0D0
:100940001BC580911702082F10E085E29BE00E94F2
:10095000C612F801E857FE4F808340911702E42F3A
:10096000F0E0E857FE4F2081809118029091190223
:10097000820F911D90931902809318024F5F40934C
:100980001702E09186012E2F30E050E04F5F5F4F5D
:100990004217530709F0F0C41092840110928301AA
:1009A000B3010E94D015AC01809185014F3F5105E4
:1009B00021F090E060E170E0DDC48D3F09F0ACC350
:1009C00080918701893009F4B8C08A3078F4833087
:1009D00001F1843020F4823009F0CEC421C0873088
:1009E00009F459C0883009F0C7C472C08A3109F4CB
:1009F000E9C08B3138F48A3009F4CFC08B3009F06C
:100A0000BBC4D4C08B3109F438C18C3109F0B4C4F3
:100A10000FC20E942502682F8DEF90E070E0AAC4FB
:100A20008091890190E081509F4F909319028093AB
:100A3000180285E29BE06FEF70E040E050E00E941A
:100A40008C1585E29BE06FEF70E040E050E00E9483
:100A50008C1585E29BE06091850140E050E00E94AA
:100A60004E156091890170E06E5F7F4F85E29BE0DB
:100A700040E050E00E948C1585E29BE060E070E071
:100A800040E050E00E948C1500911802109119026C
:100A90000E94E9023EC38DEF90E060E070E00E94AA
:100AA000D10380911C0190911D01009731F48AE1DE
:100AB00091E062E170E00E94040A809188018093D5
:100AC0001C0110921D018AE191E00E94850A54C424
:100AD0008DEF90E060E070E00E94D10340911C0136
:100AE00050911D01A9E8B1E08091880190E02CE3CC
:100AF00030E0829FF001839FF00D929FF00D112452
:100B0000E15AFD4F80E090E08F0169857A850FC042
:100B1000019611967C91119760E02C91FB01E20FF8
:100B2000F11D9F01F801219331938F0112968417D3
:100B3000950774F37A8769871FC48DEF90E060E0B2
:100B400070E00E94D1038091860190E00297B1018C
:100B50000E94D015E8E8F1E0A7E6B9E080E090E077
:100B60008D014B855C8513C02081D8012C93528167
:100B700040E02181DA01A20FB11D9D01D80112963A
:100B80003C932E931197019633960D5F1F4F861756
:100B9000970754F35C874B87EFC38DEF90E060E0DD
:100BA00070E00E94D1030E945F03E6C38DEF90E0E6
:100BB00060E070E00E94D1030E945F0318161906DE
:100BC000DCF3DAC38DEF90E060E070E00E94D103C7
:100BD000209188012530A8F530E0289DC001299D8D
:100BE000900D389D900D11246091860170E0635046
:100BF0007040865E9E4F0E94040A89E891E060E0A2
:100C000070E07C0116C08B010F5F1F4FF70141910F
:100C10007F012091880130E0289DC001299D900D21
:100C2000389D900D1124865E9E4F50E00E94720AFE
:100C3000B8018091860190E00397681779071CF34B
:100C40009BC32A3009F098C38091890180932E02BA
:100C500010922F0280918A0180933002109231020B
:100C600080918B01809332021092330280918C012B
:100C700080933402109235027FC38DEF90E060E0E4
:100C800070E00E94D10380918801853008F05CC03B
:100C900009E811E0EE24FF246801870127C070E015
:100CA000689D7001699DF00C789DF00C11242AE17B
:100CB00031E0E20EF31EB80175956795C7010E94F9
:100CC0007B0ABC010E5F1F4FD6011196BC91BA83FF
:100CD0001982F601808149815A81480F511DC7014F
:100CE0000E94050C22E030E0C20ED31E80918601E6
:100CF00090E00497609188010817190784F270E06A
:100D0000689DC001699D900D789D900D1124865EAF
:100D10009E4F0E94850A2091880130E0289DC001E5
:100D2000299D900D389D900D1124E0918601F0E0F1
:100D3000EB57FE4F608131E2639FB0011124865E64
:100D40009E4F0E94420B18C38A3009F015C3409190
:100D50008A014C831B82809189012B813C81280F61
:100D6000311D30932B0220932A0250918C015E8317
:100D70001D8280918B01AD81BE81A80FB11DB09302
:100D80002D02A0932C022115310569F4109759F416
:100D900086E292E060E070E040E050E00E94CF0F19
:100DA0000E947F0134C080913F02909140020097E1
:100DB00071F580914F0290915002009741F5E1E06A
:100DC000F0E0F0933902E093380240923E028091C5
:100DD0008F0A9091900AA091910AB091920A809303
:100DE000450290934602A0934702B0934802809137
:100DF000930A9091940AA091950AB091960A8093D3
:100E0000550290935602A0935702B09358028091D6
:100E10002A0290912B029093400280933F0280918E
:100E20002C0290912D029093500280934F02A4C205
:100E300080918801853008F05BC085E29BE06FEF10
:100E400070E040E050E00E948C1585E29BE06FEF7F
:100E500070E040E050E00E948C1585E29BE06091DC
:100E6000850140E050E00E944E1585E29BE063E082
:100E700070E040E050E00E948C1585E29BE060E06D
:100E800070E040E050E00E948C158091880190E075
:100E9000889DF001899DF00D989DF00D1124E65E6E
:100EA000FE4F6081609318021092190285E29BE068
:100EB00070E040E050E00E948C1580911802909103
:100EC0001902039620918501820F911D90931902BA
:100ED00080931802B3010E94D0156FEF70E0681B79
:100EE000790B85E29BE040E050E00E948C1544C203
:100EF0008A3009F041C227E031E030931902209393
:100F0000180285E29BE06FEF70E040E050E00E9445
:100F10008C1585E29BE06FEF70E040E050E00E94AE
:100F20008C1585E29BE06091850140E050E00E94D5
:100F30004E1585E29BE06AE070E040E050E00E94E0
:100F40008C1585E29BE060E070E040E050E00E949C
:100F50008C1580918F0A9091900AA091910AB0917E
:100F6000920A8C01107085E29BE0B80140E050E0ED
:100F70000E948C158091180290911902800F911F88
:100F8000909319028093180280918F0A9091900A91
:100F9000A091910AB091920A892F9A2FAB2FBB276B
:100FA0008C01107085E29BE0B80140E050E00E94A7
:100FB0008C158091180290911902800F911F9093C7
:100FC00019028093180280918F0A9091900AA09143
:100FD000910AB091920A0A2F10E085E29BE0B801D5
:100FE00040E050E00E948C15809118029091190207
:100FF000800F911F909319028093180220918F0AFD
:101000003091900A4091910A5091920A252F3327EE
:1010100044275527890185E29BE0B90140E050E073
:101020000E948C158091180290911902800F911FD7
:1010300090931902809318028091930A9091940AD8
:10104000A091950AB091960A8C01107085E29BE000
:10105000B80140E050E00E948C15809118029091F8
:101060001902800F911F90931902809318028091AA
:10107000930A9091940AA091950AB091960A892FAB
:101080009A2FAB2FBB278C01107085E29BE0B80133
:1010900040E050E00E948C15809118029091190256
:1010A000800F911F90931902809318028091930AE8
:1010B0009091940AA091950AB091960A0A2F10E097
:1010C00085E29BE0B80140E050E00E948C158091E1
:1010D000180290911902800F911F9093190280932A
:1010E00018022091930A3091940A4091950A5091E8
:1010F000960A252F332744275527890185E29BE04F
:10110000B90140E050E00E948C1580911802909146
:101110001902800F911FDACE909187018E3F09F05E
:10112000DCC0943809F0B0C05090880180918901EA
:10113000082F10E024503040209FC001219F900DC7
:10114000309F900D112480509F4F909319028093EF
:10115000180285E29BE06FEF70E040E050E00E94F3
:101160008C1585E29BE06FEF70E040E050E00E945C
:101170008C1585E29BE06091850140E050E00E9483
:101180004E158091860190E00497809FB001819F69
:10119000700D909F700D11246E5F7F4F85E29BE074
:1011A00040E050E00E948C1585E29BE060E070E03A
:1011B00040E050E00E948C159AE8A92E91E0B92EEB
:1011C00082E0E82EF12C980152C0D5018D915D018D
:1011D00090E0652D70E0A9012D873E870E94280DC3
:1011E0002D853E8597FF04C000E010E0690138C0FE
:1011F00004E0C02E0AE0D02E00E010E019C0F60195
:1012000061916F018091180290911902860F911DD2
:10121000909319028093180285E29BE040E050E031
:101220002D873E870E944E150F5F1F4F3E852D85EF
:101230000217130724F318C0809118029091190225
:1012400081509F4F909319028093180285E29BE092
:101250006FEF70E040E050E00E948C150F5F1F4F71
:101260000C151D054CF396010894E11CF11C8091AE
:10127000860190E00297E816F9060CF4A6CF80915B
:1012800018029091190226CE0E944C0C8FEF0E94FA
:101290005C0C8FEF0E945C0C809185010E945C0CBD
:1012A000809186010E945C0C809187010E945C0CF9
:1012B00008E811E080E090E07C0108C0D8018D9141
:1012C0008D010E945C0C0894E11CF11C8091860148
:1012D00090E0E816F90694F34FC0923021F0933075
:1012E00009F04AC029C0609188014091890190E0CD
:1012F00070E050E00E94280D8091020A8823C9F016
:101300000FEF19E080E090E07C010CC0F8016191E2
:101310008F0185E29BE040E050E00E944E1508946A
:10132000E11CF11C8091020A90E003968E159F0546
:101330006CF71092020A20C04091890160918801E7
:10134000E43031F490E070E050E00E947D0D0DC07B
:10135000F0918A01F8871F822F813885240F311D73
:10136000A90190E070E00E94B20D8091850190E0AB
:1013700060E070E00E94D10385E29BE00E9496123B
:10138000181619060CF476CA80E090E005E110E02A
:101390007C01E09EC001E19E900DF09E900D112415
:1013A000865E9E4F0E948C0B0894E11CF11C35E078
:1013B000E316F10471F70E949E012E960FB6F89481
:1013C000DEBF0FBECDBFCF91DF911F910F91FF9078
:1013D000EF90DF90CF90BF90AF909F908F907F90D5
:1013E0006F905F904F903F902F900895CF93DF9331
:1013F000CAE1D2E0CE010E94170ECE0104960E94EF
:10140000170EDF91CF910895EF92FF920F931F93E4
:10141000DF93CF9300D0CDB7DEB77C018B01CB013A
:1014200069837A830E942616D7011B968C931B979B
:101430001C969C93000F111FC8010E942616F701ED
:1014400085839683C8010E942616D70117968C9330
:10145000179718969C93C8010E942616F70181875A
:101460009287698162837A81738380E090E020E0D3
:1014700032E01EC0D7011B96ED91FC911C97E80F3E
:10148000F91F482F4F5F4083AC01440F551F15963D
:10149000ED91FC911697E40FF51F31832083179689
:1014A000ED91FC911897E40FF51F3183208301968D
:1014B000F7014281538184179507E4F21082148268
:1014C0000E940112D7011D966D937D938D939C937D
:1014D00050970F900F90CF91DF911F910F91FF9038
:1014E000EF900895DC011B96ED91FC911C97E60F9F
:1014F000F71F40830895DC011B96ED91FC911C972A
:10150000E60FF71F808190E00895EF92FF920F930E
:101510001F93CF93DF937C01C0E0D0E027C0CE01C2
:10152000880F991FD70115960D911C911697080FDA
:10153000191F1B96ED91FC911C97EC0FFD1F8081EC
:1015400090E064E270E042E050E00E94280DF3E099
:10155000880F991FFA95E1F7F8019183808369E17B
:1015600070E080E090E00E9435122196D70112963B
:101570008D919C911397C817D9078CF2DF91CF9169
:101580001F910F91FF90EF900895AF92BF92CF926D
:10159000DF92EF92FF920F931F93CF93DF936C0133
:1015A000DC0112968D919C911397EC01CC0FDD1FFD
:1015B000C80FD91F8E010C5F1F4FCB55DE4F0E9405
:1015C0004C0C8FEF0E945C0C8FEF0E945C0C8EEF36
:1015D0000E945C0C802F0E945C0C83E80E945C0CD3
:1015E0008EE10E945C0C82E00E945C0C00E010E046
:1015F0002CC0C801880F991FD6011596ED91FC915A
:101600001697E80FF91FE080F18093E0F694E794D5
:101610009A95E1F7AF2CBB24A7FCBA941B96ED91E9
:10162000FC911C97E00FF11F8081C80FD11DCE0DDA
:10163000D11DCA0DDB1D0E945C0C8E2D0E945C0C1E
:101640008A2D0E945C0C0F5F1F4FF60182819381EF
:101650000817190774F2CE0160E071E00E94D015FE
:1016600080950E945C0C80E090E00E94380CDF9135
:10167000CF911F910F91FF90EF90DF90CF90BF908F
:10168000AF9008950F931F93CF93DF93EC01CB019D
:1016900061E270E00E94D0158B010F5F1F4F0E9426
:1016A00001126D877E878F87988B20E030E028C0FD
:1016B000B901660F771FEF81F885E60FF71F80816C
:1016C0009181ED81FE81E60FF71F40815181E9850F
:1016D000FA854817590728F4E60FF71F841B950B66
:1016E00006C0E60FF71FBA01681B790BCB01B801E2
:1016F0000E94BC156F5F7F4F718360832F5F3F4FE8
:101700008A819B81281739079CF281E08883DF91C9
:10171000CF911F910F910895CF92DF92EF92FF9298
:101720000F931F93CF93DF93EC018881882309F4F3
:1017300063C00A811B810E9401122D853E854F8561
:101740005889621B730B840B950B613271058105FF
:10175000910588F30E9401126D877E878F87988B91
:1017600080E090E03CC0AC01440F551FEF81F8854C
:10177000E40FF51FC080D180ED81FE81E40FF51FDD
:10178000E080F18096012E193F0981F069857A8504
:10179000121613069CF4460F571FDA014D915C9107
:1017A0001197241735072CF4D182C08201501040C4
:1017B00015C04E0D5F1D5183408310C0460F571F4B
:1017C000DA014D915C911197309521953F4F241787
:1017D000350754F3E41AF50AF182E08201962A8172
:1017E0003B81821793070CF4BECF101611060CF044
:1017F0001882CE010E94C50ADF91CF911F910F91EF
:10180000FF90EF90DF90CF900895FC01228133810B
:1018100080E090E019C0A385B485A80FB91FAC91F2
:10182000B0E0A617B70779F4880F991F0780F085F5
:10183000E02DE80FF91F33E0440F551F3A95E1F70B
:1018400051834083089501968217930724F30895E6
:10185000E9ECF0E080818F7E8083808188608083E6
:1018600080818F7780831092620A1092610A0895B6
:10187000E9ECF0E08081877F8083808180688083CD
:101880008081806180831092640A1092630A1092B2
:10189000600A10925F0A0895E9ECF0E080818F7E83
:1018A000808380818860808380818F77808310929D
:1018B000620A1092610A08959091C80095FFFCCFCA
:1018C0008093CE0008952091610A3091620AF90157
:1018D000E15EF54F80832F5F3F4F3093620A209384
:1018E000610A9091C80095FFFCCF8093CE000895C7
:1018F0001F920F920FB60F9211242F938F939F93E5
:10190000EF93FF938091630A9091640A2091CE0037
:10191000FC01E15CF54F208301969093640A80936B
:10192000630AFF91EF919F918F912F910F900FBEBE
:101930000F901F9018951F93DF93CF930F92CDB701
:10194000DEB7198210E01CC02F5F3F4F43E02A3EF4
:10195000340729F41AC020E030E0A12FB0E06981FB
:101960004091630A5091640AFD01E60FF11DE417EE
:10197000F50751F326C02091FF092F3F81F11F5F2A
:10198000298130E02817390734F3898180E092E01B
:1019900007C0E92FF0E0E150F64F2081820F9F5FF2
:1019A00029819217B0F390E021E030E08F3F91055C
:1019B00011F020E030E0C9010F90CF91DF911F912D
:1019C0000895E9812981F0E0E150F64FA15CB54F1F
:1019D000A20FB11D2C9120832981222361F229813C
:1019E0002F5F2983CDCF9B01AC0163E0220F331F12
:1019F000441F551F6A95D1F760E074E284EF90E0D0
:101A00000E940516DA01C9010197A109B109892FC0
:101A10009A2FAB2FBB27A7FDBA958093CD002150FD
:101A20002093CC00E8ECF0E080818260808310920B
:101A3000640A1092630A1092600A10925F0A109270
:101A4000620A1092610A80E090E00E94380C0895CA
:101A5000EF92FF920F931F93CF93DF938C017B0143
:101A6000EA010E94280C8FEF0E94630C8FEF0E9406
:101A7000630C802F0E94630C84E00E94630C82E060
:101A80000E94630C8E2D0E94630C8C2F0E94630CAD
:101A9000C80106968E0D9F1D8C0F9D1F60E071E0A2
:101AA0000E94D01580950E94630CC8010E94380CDA
:101AB000CE0106960E949B0C18161906A4F480917C
:101AC000030A8093650A1092660A8091040AC13065
:101AD000D10519F4282F30E008C03091050A20E024
:101AE000280F311D02C02FEF3FEFC901DF91CF91C9
:101AF0001F910F91FF90EF900895FF920F931F9306
:101B0000CF93DF93EC018B01F42E0E94280C8FEF12
:101B10000E94630C8FEF0E94630C8C2F0E94630C59
:101B200084E00E94630C83E00E94630C802F0E947B
:101B3000630C8F2D0E94630CCE010796800F911FBE
:101B40008F0D911D60E071E00E94D01580950E947C
:101B5000630CCE010E94380CDF91CF911F910F9141
:101B6000FF900895AF92BF92DF92EF92FF920F9392
:101B70001F93DF93CF930F92CDB7DEB75C018B013C
:101B8000D42E59830E94280C5981E52EFF248FEF13
:101B90000E94630C8FEF0E94630C8A2D0E94630CDD
:101BA00085E00E94630C83E00E94630C802F0E94FA
:101BB000630C8D2D0E94630C8E2D0E94630CC50159
:101BC0000896800F911F8D0D911D8E0D9F1D809584
:101BD0000E94630CC5010E94380C0F90CF91DF91D9
:101BE0001F910F91FF90EF90DF90BF90AF900895FD
:101BF0002FB7F89482E0809380008AE1809381007F
:101C000088EB9BE0909389008093880090938B00F1
:101C100080938A0080E49CE99093870080938600FB
:101C2000EFE6F0E08081887F80832FBF0895FC017C
:101C300010828FEF818308950F931F93CF93DF93CB
:101C4000EC018B01CA01F9019B012C50304022307C
:101C50003105C8F520E130E0B9010E94D0156A8352
:101C6000CF01B9010E94D0156B8308838FEF898360
:101C7000802F60E00E941E11888161E00E94FA10AE
:101C80008091670A882331F48091680A882311F4CF
:101C90000E94F80D88818D3049F481E08093670AB5
:101CA000809180008F7380688093800088818C3061
:101CB00061F481E08093680A809180008F7C80626B
:101CC0008093800002C080E001C081E0DF91CF916D
:101CD0001F910F91089540E252E020E639E00E9402
:101CE0001C0E0895CF93DF93EC0188818D3059F459
:101CF0001092670A809180008F73809380008881A2
:101D000060E00E94FA1088818C3059F41092680AC1
:101D1000809180008F7C80938000888160E00E94A9
:101D2000FA10DF91CF910895FC0181E0643F7807BC
:101D30002CF089E0653C780724F405C064EF71E07D
:101D400002C064EC79E0660F771F80818D3021F44A
:101D5000709389006093880080818C3021F47093A7
:101D60008B0060938A000895FC0180818D3021F4FE
:101D700081E09091670A05C08C3039F481E0909140
:101D8000680A992319F480E0089580E008951F926D
:101D90000F920FB60F9211242F933F934F935F939F
:101DA0006F937F938F939F93AF93BF93EF93FF9323
:101DB00080918E0A87FF05C01092850010928400E2
:101DC0002BC020918E0A332727FD30958091690A18
:101DD00090E02817390704F580918E0A992787FD2E
:101DE0009095FC01EE0FFF1FE80FF91FE659F54F24
:101DF000808186FF11C080918E0A992787FD90957A
:101E0000FC01EE0FFF1FE80FF91FE659F54F808127
:101E10008F7360E00E941E1180918E0A8F5F809305
:101E20008E0A20918E0A332727FD30958091690A0A
:101E300090E0281739070CF04EC080918E0A8C3044
:101E40000CF049C0809184009091850020918E0A09
:101E5000332727FD3095F901EE0FFF1FE20FF31F27
:101E6000E659F54F21813281820F931F90938900AB
:101E70008093880080918E0A992787FD9095FC01B8
:101E8000EE0FFF1FE80FF91FE659F54F808186FF1F
:101E90002BC080918E0A992787FD9095FC01EE0F4B
:101EA000FF1FE80FF91FE659F54F80818F7361E03E
:101EB0000E941E1119C080E49CE905C08091840035
:101EC00090918500049690938900809388008FEF0D
:101ED00080938E0A09C080918400909185002CE93E
:101EE0008434920740F3EACFFF91EF91BF91AF9115
:101EF0009F918F917F916F915F914F913F912F9122
:101F00000F900FBE0F901F901895CF93DF93EB01AA
:101F1000FC017183608377FD0BC082E160E00E9469
:101F20001E1182E061E00E941E118EE0BE010DC014
:101F300082E060E00E941E1182E161E00E941E11B9
:101F4000662777276C1B7D0B8EE00E94A110DF9126
:101F5000CF910895CF93DF93EB01FC0173836283EC
:101F600077FD0BC083E160E00E941E1181E061E01B
:101F70000E941E118FE0BE010DC081E060E00E9452
:101F80001E1183E161E00E941E11662777276C1BFA
:101F90007D0B8FE00E94A110DF91CF9108950F93E8
:101FA0001F93CF93DF93EC018A010E94850FCE012E
:101FB000B8010E94AA0FDF91CF911F910F91089550
:101FC0001F920F920FB60F9211242F933F934F93AE
:101FD0005F936F938F939F93AF93BF93EF93FF9311
:101FE00066B1262F30E04091970A50E042275327F0
:101FF00044FF2AC0C9018072907095958795F901B8
:10200000E071F0708E179F0761F48091930A9091B0
:10201000940AA091950AB091960A0196A11DB11D4E
:102020000BC08091930A9091940AA091950AB09167
:10203000960A0197A109B1098093930A9093940A93
:10204000A093950AB093960A46FF29C0C9018078EB
:10205000907095958795207430708217930761F47E
:1020600080918F0A9091900AA091910AB091920A62
:102070000196A11DB11D0BC080918F0A9091900A0D
:10208000A091910AB091920A0197A109B109809398
:102090008F0A9093900AA093910AB093920A60934A
:1020A000970AFF91EF91BF91AF919F918F916F919F
:1020B0005F914F913F912F910F900FBE0F901F9006
:1020C0001895E8E6F0E0808184608083EDE6F0E03A
:1020D00080818065808386B18093970A08951092ED
:1020E0008F0A1092900A1092910A1092920A1092FE
:1020F000930A1092940A1092950A1092960A0895E3
:102100008E3008F08E508770909107019295990F4C
:10211000990F907C982B90937C0080917A0080643A
:1021200080937A0080917A0086FDFCCF2091780020
:1021300030917900932F80E030E0282B392BC901B2
:1021400008951F93CF93DF93182FEB0161E00E9456
:10215000FA10E12FF0E0E652FF4FE491E33051F442
:1021600080918000806880938000D0938900C09324
:1021700088003CC0E43051F48091800080628093FC
:102180008000D0938B00C0938A0030C0E13039F4D6
:10219000209729F184B5806884BDC7BD27C0E2308F
:1021A00039F42097E1F084B5806284BDC8BD1EC0BB
:1021B000E63041F48091B00080688093B000C09315
:1021C000B30014C0E73041F48091B0008062809386
:1021D000B000C093B4000AC0C038D1051CF4812FF0
:1021E00060E002C0812F61E00E941E11DF91CF915B
:1021F0001F91089590E0FC01E654FF4F2491FC01EB
:10220000E656FF4FE491EE23C1F0F0E0EE0FFF1F22
:10221000E458FF4F85919491DC01662341F49FB708
:10222000F8948C91209582238C939FBF08959FB73B
:10223000F8948C91822B8C939FBF089590E0FC01C1
:10224000E652FF4F2491FC01E654FF4F449186561D
:102250009F4FFC018491882309F441C0222331F16E
:10226000233021F4909180009F7705C0243031F411
:10227000909180009F7D9093800018C0213019F4C8
:1022800094B59F7704C0223021F494B59F7D94BD0E
:102290000DC0263021F49091B0009F7705C0273003
:1022A00029F49091B0009F7D9093B000E82FF0E06A
:1022B000EE0FFF1FEA57FF4F25913491D901662396
:1022C00041F49FB7F8948C91409584238C939FBFE1
:1022D00008959FB7F8948C91842B8C939FBF089599
:1022E00090E0FC01E652FF4F2491FC01E654FF4FC1
:1022F000449186569F4FFC0184918823B1F122239B
:1023000031F1233021F4909180009F7705C0243073
:1023100031F4909180009F7D9093800018C021300F
:1023200019F494B59F7704C0223021F494B59F7DB1
:1023300094BD0DC0263021F49091B0009F7705C068
:10234000273029F49091B0009F7D9093B000E82F42
:10235000F0E0EE0FFF1FE057FF4F25913491D901B8
:102360008C91842321E030E011F420E030E0C901B9
:1023700008951F920F920FB60F9211242F933F933F
:102380008F939F93AF93BF9380919C0A90919D0AE6
:10239000A0919E0AB0919F0A3091A00A0196A11DBA
:1023A000B11D232F2D5F2D3720F02D570196A11D34
:1023B000B11D2093A00A80939C0A90939D0AA0933C
:1023C0009E0AB0939F0A8091980A9091990AA091D1
:1023D0009A0AB0919B0A0196A11DB11D8093980A9B
:1023E0009093990AA0939A0AB0939B0ABF91AF91D8
:1023F0009F918F913F912F910F900FBE0F901F9043
:1024000018958FB7F89420919C0A30919D0A4091BD
:102410009E0A50919F0A8FBFB901CA0108959FB7C4
:10242000F8942091980A3091990A40919A0A509113
:102430009B0A86B5A89B06C08F3F21F02F5F3F4FB8
:102440004F4F5F4F9FBF542F432F322F2227280F0C
:10245000311D411D511D82E0220F331F441F551FA6
:102460008A95D1F7B901CA010895EF92FF920F93AF
:102470001F93CF93DF937B018C010E940F12EB011E
:102480000FC00E940F126C1B7D0B83E0683E780723
:1024900038F00894E108F10801091109C851DC4F2E
:1024A000E114F1040105110561F7DF91CF911F914E
:1024B0000F91FF90EF900895789484B5826084BD69
:1024C00084B5816084BD85B5826085BD85B5816038
:1024D00085BDEEE6F0E0808181608083E1E8F0E098
:1024E000808182608083808181608083E0E8F0E089
:1024F000808181608083E1EBF0E080818460808373
:10250000E0EBF0E0808181608083EAE7F0E08081A9
:102510008460808380818260808380818160808309
:102520008081806880831092C1000895FC0122811F
:102530003381F901E058FF4F8081918180589F4F8E
:102540002E573F4FF90120813181821B930B60E8A8
:1025500070E00E94D0150895FC0182819381FC01F6
:10256000EE57FF4F20813181FC01E058FF4F408141
:1025700051814217530731F0820F931FFC012081D4
:1025800030E002C02FEF3FEFC9010895DC01129641
:102590002D913C911397F901EE57FF4F8081918166
:1025A000D901A058BF4F4D915C9111974817590719
:1025B00069F0280F391FD9012C91019660E870E06D
:1025C0000E94D0159183808330E002C02FEF3FEF4F
:1025D000C9010895DC0112968D919C911397FC011D
:1025E000E058FF4F8E579F4FDC018D919C911197C2
:1025F000918380830895FC01A085B18521898C9108
:1026000090E0022E02C0959587950A94E2F780FF2C
:10261000F6CF0484F585E02D608308951F93CF9352
:10262000DF93182F9B01EB01C058DF4FE881F98140
:10263000CF01019660E870E00E94D015AC01D9018D
:10264000AE57BF4F8D919C9111974817590729F0AC
:10265000E20FF31F108359834883DF91CF911F91BD
:1026600008951F920F920FB60F9211242F933F934C
:102670004F935F936F937F938F939F93AF93BF938A
:10268000EF93FF938091C60061EA7AE00E940E13F7
:10269000FF91EF91BF91AF919F918F917F916F913A
:1026A0005F914F913F912F910F900FBE0F901F9010
:1026B00018958F929F92AF92BF92DF92EF92FF9206
:1026C0000F931F93CF93DF93EC017A018B01413479
:1026D00082E458078FE0680780E078070CF07DC03F
:1026E00060E874E88EE190E0A80197010E94051669
:1026F0002150304040405040CA01B90122E030E052
:1027000040E050E00E94051649015A01209530959D
:102710004095509594E0220F331F441F551F9A9502
:10272000D1F760E074E284EF90E00E940516CA01E0
:10273000B9012FEF30E040E050E00E949D15A80164
:1027400097010E940516C90181509F4F181619065E
:102750001CF4D22EDA9403C0DD24D394D21A60E0A4
:1027600079E08DE390E0A80197010E9405162150C1
:10277000304040405040CA01B90122E030E040E022
:1027800050E00E940516209530954095509583E0C5
:10279000220F331F441F551F8A95D1F760E074E262
:1027A00084EF90E00E940516CA01B9012FEF30E0D6
:1027B00040E050E00E949D15A80197010E94051677
:1027C000C90181509F4F181619061CF4822F8150A1
:1027D00002C081E0821B8D1500F5E885F98581E056
:1027E00090E00A8802C0880F991F0A94E2F780835C
:1027F00060E079E08DE390E0A80197010E94051662
:102800002150304040405040CA01B90122E030E040
:1028100040E050E00E94051604C0E885F98510826A
:102820009401EC81FD813083EE81FF812083EA8574
:10283000FB85408181E090E09C010E8402C0220F64
:10284000331F0A94E2F7422B4083EA85FB854081DF
:102850009C010F8402C0220F331F0A94E2F7422B1F
:102860004083EA85FB852081088802C0880F991F74
:102870000A94E2F7282B2083DF91CF911F910F91CB
:10288000FF90EF90DF90BF90AF909F908F90089552
:102890008CE091E09093260B8093250B81EA9AE0DF
:1028A0009093280B8093270B85EC90E090932A0B54
:1028B0008093290B84EC90E090932C0B80932B0B4E
:1028C00080EC90E090932E0B80932D0B81EC90E0A8
:1028D0009093300B80932F0B86EC90E09093320B0B
:1028E0008093310B84E08093330B83E08093340B2F
:1028F00087E08093350B85E08093360B81E08093F1
:10290000370B08950F931F93CF93DF93EC01062F9E
:10291000172F07C0E881F9810190F081E02DCE01E9
:102920000995F80161918F016623A1F7DF91CF919D
:102930001F910F910895EF92FF920F931F93CF93E2
:10294000DF937C01EB018A010BC06991D701ED9106
:10295000FC910190F081E02DC701099501501040D4
:102960000115110591F7DF91CF911F910F91FF9004
:10297000EF9008956F927F928F929F92AF92BF9245
:10298000CF92DF92EF92FF920F931F93DF93CF933B
:10299000CDB7DEB7A0970FB6F894DEBF0FBECDBFA0
:1029A0005C01CB01BA01611571058105910551F4F6
:1029B000C50140E350E060E070E020E030E00E94BC
:1029C000561548C06E010894C11CD11CEE24FF248A
:1029D0008701622E772488249924A40193010E9400
:1029E000E315F60161936F010894E11CF11C011DD0
:1029F000111DB901CA01611571058105910569F7BC
:102A0000D801C7010197A109B1096E010894C11C41
:102A1000D11CC80ED91E19C0F60140814A3010F4ED
:102A2000405D01C0495C552747FD5095652F752FC6
:102A3000C50120E030E00E9456150894E108F10835
:102A4000010911090894C108D108E114F104010534
:102A5000110511F7A0960FB6F894DEBF0FBECDBFDB
:102A6000CF91DF911F910F91FF90EF90DF90CF906A
:102A7000BF90AF909F908F907F906F900895211599
:102A8000310549F4DC01ED91FC910190F081E02DDC
:102A9000642F099508950E94BA1408959A01462F4B
:102AA00050E060E070E00E943F150895EF92FF92C1
:102AB0000F931F93CF93DF93EC017A018B012115C4
:102AC000310541F4E881F9810190F081E02D642F16
:102AD00009951BC02A303105B1F477FF10C04DE2D3
:102AE00050E060E070E020E030E00E945615109564
:102AF0000095F094E094E11CF11C011D111DCE0124
:102B0000B801A7012AE00E94BA14DF91CF911F916A
:102B10000F91FF90EF9008959A01FB01AF01662796
:102B200057FD6095762F0E94561508950E945C12FD
:102B30000E940C020E941404FDCF629FD001739F7B
:102B4000F001829FE00DF11D649FE00DF11D929F49
:102B5000F00D839FF00D749FF00D659FF00D992788
:102B6000729FB00DE11DF91F639FB00DE11DF91FAC
:102B7000BD01CF0111240895AA1BBB1B51E107C061
:102B8000AA1FBB1FA617B70710F0A61BB70B881FFD
:102B9000991F5A95A9F780959095BC01CD0108958C
:102BA00097FB092E07260AD077FD04D0E5DF06D073
:102BB00000201AF4709561957F4F0895F6F790956F
:102BC00081959F4F0895A1E21A2EAA1BBB1BFD0100
:102BD0000DC0AA1FBB1FEE1FFF1FA217B307E407FC
:102BE000F50720F0A21BB30BE40BF50B661F771F54
:102BF000881F991F1A9469F7609570958095909534
:102C00009B01AC01BD01CF01089597FB092E05265C
:102C10000ED057FD04D0D7DF0AD0001C38F45095F1
:102C20004095309521953F4F4F4F5F4F0895F6F7F0
:102C300090958095709561957F4F8F4F9F4F089528
:102C4000EE0FFF1F0590F491E02D0994CF93DF93D1
:102C50008230910510F482E090E0E0913A0BF0911F
:102C60003B0B40E050E020E030E026C06081718105
:102C700068177907E0F06817790781F482819381FA
:102C80002115310531F0D90113969C938E9312973B
:102C90002BC090933B0B80933A0B26C041155105F6
:102CA00019F06417750718F4AB01E901DF019F0102
:102CB00072816381E72FF62F3097C1F641155105D8
:102CC00001F1481B590B4430510580F412968D9147
:102CD0009C911397209719F09B838A8304C090934B
:102CE0003B0B80933A0BFD01329646C0FD01E40F89
:102CF000F51F819391934250504011965C934E93EF
:102D00003BC02091380B3091390B2115310541F42E
:102D100020910201309103013093390B2093380B3D
:102D200020910401309105012115310541F42DB7A1
:102D30003EB74091000150910101241B350BE091F9
:102D4000380BF091390BE217F307A0F42E1B3F0B61
:102D50002817390778F0AC014E5F5F4F241735070D
:102D600048F04E0F5F1F5093390B4093380B8193FF
:102D7000919302C0E0E0F0E0CF01DF91CF910895A0
:102D8000CF93DF93009709F491C0FC01329713822F
:102D9000128260913A0B70913B0B6115710581F4C1
:102DA00020813181280F391F8091380B9091390B88
:102DB0008217930799F5F093390BE093380B76C09F
:102DC000DB0180E090E002C0CD01D901AE17BF0762
:102DD00048F412962D913C91139721153105A1F7D6
:102DE000CD0121C0B383A283EF01499159919E0186
:102DF000240F351FA217B30779F42D913C91119739
:102E0000240F351F2E5F3F4F3183208312962D9163
:102E10003C91139733832283009729F4F0933B0B63
:102E2000E0933A0B43C0DC011396FC93EE931297A8
:102E30004D915D91A40FB51FEA17FB0769F420813E
:102E40003181240F351F2E5F3F4FEC0139832883DA
:102E5000228133813B832A83E0E0F0E002C0FB0162
:102E6000BC01DB0112968D919C9113970097B9F7E5
:102E70009B012E5F3F4F8D919C911197820F931F65
:102E80004091380B5091390B4817590779F4309716
:102E900029F410923B0B10923A0B02C0138212825B
:102EA000225030403093390B2093380BDF91CF9173
:062EB0000895F894FFCF25
:102EB60020003C0B0000010100000000FB12821400
:0A2EC6009B149612C612EA12AC1219
:00000001FF
